:100000000C945A000C9477000C9477000C947700B1
:100010000C9477000C9477000C9477000C94770084
:100020000C9477000C9477000C9477000C94770074
:100030000C9477000C9477000C9477000C94770064
:100040000C944B010C9477000C9477000C9477007F
:100050000C9477000C9477000C9477000C94770044
:100060000C9477000C947700000024272A000025C8
:10007000282B000023262904040404040404040299
:100080000202020202030303030303010204081035
:100090002040800102040810200102040810200002
:1000A0000000070002010000030406000000000039
:1000B0000000000011241FBECFEFD4E0DEBFCDBF93
:1000C00011E0A0E0B1E0E2EAF5E002C005900D9297
:1000D000A031B107D9F711E0A0E1B1E001C01D9254
:1000E000AA31B107E1F70E9444010C94D0020C94AC
:1000F000000061E0809100010E94F90161E08091BF
:1001000002010E94F90161E0809104010E94F9015D
:1001100061E0809106010E94F90161E0809108018F
:100120000E94F90161E080910A010E94F90161E0F9
:1001300080910C010E94F90161E080910E010E9402
:10014000F90161E0809100010E94630261E0809109
:1001500002010E94630261E0809104010E94630237
:1001600061E0809106010E94630260E080910801D5
:100170000E94630260E080910A010E94630260E0D5
:1001800080910C010E94630260E080910E010E9448
:1001900063020895109213011092120168EE73E049
:1001A00080E090E00E9488018091120190911301FB
:1001B00001969093130180931201CC977CF30895DC
:1001C00010921501109214010E94CA00809114012E
:1001D0009091150101969093150180931401CC978D
:1001E0009CF308958091100190911101892B09F0E1
:1001F0004AC081E090E0909311018093100161E08A
:10020000809108010E9463020E94E00060E08091FA
:1002100000010E94630260E0809108010E94630275
:1002200061E080910A010E9463020E94E00060E0A8
:10023000809102010E94630260E080910A010E94A5
:10024000630261E080910C010E9463020E94E00061
:1002500060E0809104010E94630260E080910C01E3
:100260000E94630261E080910E010E9463020E947D
:10027000E00060E0809106010E94630260E08091EE
:100280000E010E94630208950E94B7010E94790046
:100290000E94F200FDCF1F920F920FB60F92112411
:1002A0008F939F93AF93BF93809116019091170105
:1002B000A0911801B09119010196A11DB11D809363
:1002C000160190931701A0931801B0931901BF91E3
:1002D000AF919F918F910F900FBE0F901F90189527
:1002E0006091160170911701809118019091190188
:1002F00027E0660F771F881F991F2A95D1F72DE7F2
:1003000030E040E050E00E94AE02CA01B901089519
:10031000AF92BF92CF92DF92EF92FF920F931F9313
:100320005B016C010E9470017B018C010E947001D5
:100330006E197F09800B910B6A157B058C059D0555
:10034000A8F31F910F91FF90EF90DF90CF90BF9097
:10035000AF900895019751F0880F991F880F991F4A
:1003600002972FB7F8940197F1F72FBF089578946B
:100370001092160110921701109218011092190193
:1003800084B5826084BD84B5816084BD85B582609A
:1003900085BD85B5816085BDEEE6F0E08081816038
:1003A0008083E1E8F0E080818260808380818160E9
:1003B0008083E0E8F0E0808181608083E1EBF0E021
:1003C000808184608083E0EBF0E0808181608083C5
:1003D000EAE7F0E0808184608083808182608083AE
:1003E0008081816080838081806880831092C100D9
:1003F0000895282F3327C90185579F4FFC019491F9
:1004000029583F4FF9018491882381F0E82FFF2775
:10041000E859FF4FE491FF27662329F480819095E6
:100420008923808308958081892B80830895482FB4
:100430005527CA0181569F4FFC012491CA01855757
:100440009F4FFC01949149585F4FFA013491332337
:1004500019F480E090E00895222331F1233021F453
:10046000809180008F7705C0243031F48091800026
:100470008F7D8093800018C0213019F484B58F7768
:1004800004C0223021F484B58F7D84BD0DC0263098
:1004900021F48091B0008F7705C0273029F4809136
:1004A000B0008F7D8093B000E32FFF27EE58FF4F01
:1004B000E491FF27808120E030E0892311F021E0E2
:1004C00030E0C9010895482F5527CA0181569F4F32
:1004D000FC012491CA0185579F4FFC019491495812
:1004E0005F4FFA0134913323C1F1222331F12330DC
:1004F00021F4809180008F7705C0243031F4809101
:1005000080008F7D8093800018C0213019F484B55D
:100510008F7704C0223021F484B58F7D84BD0DC057
:10052000263021F48091B0008F7705C0273029F460
:100530008091B0008F7D8093B000E32FFF27E359B7
:10054000FF4FE491FF27662329F48081909589234A
:10055000808308958081892B80830895A1E21A2EDB
:10056000AA1BBB1BFD010DC0AA1FBB1FEE1FFF1F57
:10057000A217B307E407F50720F0A21BB30BE40BA7
:10058000F50B661F771F881F991F1A9469F76095EE
:100590007095809590959B01AC01BD01CF010895A8
:0205A000FFCF8B
:1005A200060007000800090002000300040005001D
:00000001FF
